BL51 BANKED LINKER/LOCATER V5.03                                                        10/07/2003  00:07:48  PAGE 1


BL51 BANKED LINKER/LOCATER V5.03, INVOKED BY:
F:\WINSOFT\KEIL\C51\BIN\BL51.EXE e51pro.obj, AT89C51PRO.obj TO E51p


MEMORY MODEL: SMALL


INPUT MODULES INCLUDED:
  e51pro.obj (E51PRO)
  AT89C51PRO.obj (AT89C51PRO)
  F:\WINSOFT\KEIL\C51\LIB\C51S.LIB (?C_STARTUP)
  F:\WINSOFT\KEIL\C51\LIB\C51S.LIB (?C?ULCMP)


LINK MAP OF MODULE:  E51p (E51PRO)


            TYPE    BASE      LENGTH    RELOCATION   SEGMENT NAME
            -----------------------------------------------------

            * * * * * * *   D A T A   M E M O R Y   * * * * * * *
            REG     0000H     0008H     ABSOLUTE     "REG BANK 0"
            DATA    0008H     0014H     UNIT         ?DT?E51PRO
            DATA    001CH     0004H     UNIT         _DATA_GROUP_
            IDATA   0020H     0001H     UNIT         ?STACK

            * * * * * * *   C O D E   M E M O R Y   * * * * * * *
            CODE    0000H     0003H     ABSOLUTE     
            CODE    0003H     003EH     UNIT         ?PR?_DELAY?E51PRO
            CODE    0041H     003AH     UNIT         ?PR?MAIN?E51PRO
            CODE    007BH     0037H     UNIT         ?PR?PRO00?AT89C51PRO
            CODE    00B2H     0031H     UNIT         ?PR?WAITCOMM?E51PRO
            CODE    00E3H     0015H     UNIT         ?PR?SENDDATA?E51PRO
            CODE    00F8H     0011H     UNIT         ?C?LIB_CODE
            CODE    0109H     000CH     UNIT         ?C_C51STARTUP
            CODE    0115H     0003H     UNIT         ?PR?RSTPRO00?AT89C51PRO
            CODE    0118H     0003H     UNIT         ?PR?READSIGN00?AT89C51PRO
            CODE    011BH     0003H     UNIT         ?PR?ERASE00?AT89C51PRO
            CODE    011EH     0003H     UNIT         ?PR?WRITE00?AT89C51PRO
            CODE    0121H     0003H     UNIT         ?PR?READ00?AT89C51PRO
            CODE    0124H     0003H     UNIT         ?PR?LOCKBIT00?AT89C51PRO



OVERLAY MAP OF MODULE:   E51p (E51PRO)


SEGMENT                             DATA_GROUP 
  +--> CALLED SEGMENT             START    LENGTH
-------------------------------------------------
?C_C51STARTUP                     -----    -----
  +--> ?PR?MAIN?E51PRO

?PR?MAIN?E51PRO                   -----    -----
  +--> ?PR?WAITCOMM?E51PRO
  +--> ?PR?_DELAY?E51PRO
  +--> ?PR?SENDDATA?E51PRO
  +--> ?PR?PRO00?AT89C51PRO
BL51 BANKED LINKER/LOCATER V5.03                                                      10/07/2003  00:07:48  PAGE 2



?PR?_DELAY?E51PRO                 001CH    0004H

?PR?PRO00?AT89C51PRO              -----    -----
  +--> ?PR?_DELAY?E51PRO
  +--> ?PR?RSTPRO00?AT89C51PRO
  +--> ?PR?READSIGN00?AT89C51PRO
  +--> ?PR?ERASE00?AT89C51PRO
  +--> ?PR?WRITE00?AT89C51PRO
  +--> ?PR?READ00?AT89C51PRO
  +--> ?PR?LOCKBIT00?AT89C51PRO

?PR?RSTPRO00?AT89C51PRO           -----    -----
  +--> ?PR?SENDDATA?E51PRO

?PR?READSIGN00?AT89C51PRO         -----    -----
  +--> ?PR?SENDDATA?E51PRO

?PR?ERASE00?AT89C51PRO            -----    -----
  +--> ?PR?SENDDATA?E51PRO

?PR?WRITE00?AT89C51PRO            -----    -----
  +--> ?PR?SENDDATA?E51PRO

?PR?READ00?AT89C51PRO             -----    -----
  +--> ?PR?SENDDATA?E51PRO

?PR?LOCKBIT00?AT89C51PRO          -----    -----
  +--> ?PR?SENDDATA?E51PRO



SYMBOL TABLE OF MODULE:  E51p (E51PRO)

  VALUE           TYPE          NAME
  ----------------------------------

  -------         MODULE        E51PRO
  C:0000H         SYMBOL        _ICE_DUMMY_
  C:00E3H         PUBLIC        SendData
  D:00A8H         PUBLIC        IE
  B:0098H.0       PUBLIC        RI
  B:0098H.1       PUBLIC        TI
  D:0081H         PUBLIC        SP
  C:00B2H         PUBLIC        WaitComm
  C:0041H         PUBLIC        main
  D:0099H         PUBLIC        SBUF
  D:0087H         PUBLIC        PCON
  D:0098H         PUBLIC        SCON
  D:0089H         PUBLIC        TMOD
  D:0088H         PUBLIC        TCON
  D:0008H         PUBLIC        nAddress
  D:000AH         PUBLIC        ComBuf
  D:008DH         PUBLIC        TH1
  C:000BH         PUBLIC        _Delay
  D:008BH         PUBLIC        TL1
  B:0088H.6       PUBLIC        TR1
BL51 BANKED LINKER/LOCATER V5.03                                                      10/07/2003  00:07:48  PAGE 3


  -------         PROC          L?0030
  -------         ENDPROC       L?0030
  -------         PROC          _DELAY
  D:001CH         SYMBOL        nTimer
  C:000BH         LINE#         10
  C:0013H         LINE#         11
  C:0013H         LINE#         12
  C:0026H         LINE#         13
  C:0026H         LINE#         14
  C:0040H         LINE#         15
  -------         ENDPROC       _DELAY
  -------         PROC          WAITCOMM
  -------         DO            
  D:0007H         SYMBOL        n
  D:0004H         SYMBOL        nTimeOut
  -------         ENDDO         
  C:00B2H         LINE#         17
  C:00B2H         LINE#         18
  C:00B2H         LINE#         19
  C:00B4H         LINE#         21
  C:00B7H         LINE#         22
  C:00B7H         LINE#         23
  C:00B7H         LINE#         24
  C:00B7H         LINE#         26
  C:00BFH         LINE#         27
  C:00BFH         LINE#         28
  C:00C2H         LINE#         29
  C:00C5H         LINE#         30
  C:00C5H         LINE#         31
  C:00CEH         LINE#         32
  C:00CFH         LINE#         33
  C:00D4H         LINE#         34
  C:00D6H         LINE#         35
  C:00DCH         LINE#         36
  C:00DEH         LINE#         37
  C:00E1H         LINE#         38
  C:00E2H         LINE#         39
  -------         ENDPROC       WAITCOMM
  -------         PROC          SENDDATA
  -------         DO            
  D:0007H         SYMBOL        n
  -------         ENDDO         
  C:00E3H         LINE#         41
  C:00E3H         LINE#         42
  C:00E3H         LINE#         43
  C:00E5H         LINE#         44
  C:00E5H         LINE#         45
  C:00E5H         LINE#         46
  C:00E7H         LINE#         47
  C:00EEH         LINE#         48
  C:00F1H         LINE#         49
  C:00F3H         LINE#         50
  C:00F7H         LINE#         51
  -------         ENDPROC       SENDDATA
  -------         PROC          MAIN
  C:0041H         LINE#         56
  C:0041H         LINE#         57
BL51 BANKED LINKER/LOCATER V5.03                                                      10/07/2003  00:07:48  PAGE 4


  C:0041H         LINE#         58
  C:0044H         LINE#         59
  C:0047H         LINE#         60
  C:0049H         LINE#         61
  C:004CH         LINE#         62
  C:004EH         LINE#         65
  C:0051H         LINE#         66
  C:0054H         LINE#         67
  C:0057H         LINE#         70
  C:005AH         LINE#         71
  C:005CH         LINE#         72
  C:005CH         LINE#         73
  C:005CH         LINE#         74
  C:0061H         LINE#         75
  C:0061H         LINE#         76
  C:0064H         LINE#         77
  C:0067H         LINE#         78
  C:006AH         LINE#         79
  C:006DH         LINE#         80
  C:0070H         LINE#         81
  C:0072H         LINE#         82
  C:0072H         LINE#         83
  C:0076H         LINE#         84
  C:0076H         LINE#         85
  C:0076H         LINE#         86
  C:0079H         LINE#         87
  -------         ENDPROC       MAIN
  -------         ENDMOD        E51PRO

  -------         MODULE        AT89C51PRO
  C:0000H         SYMBOL        _ICE_DUMMY_
  C:0124H         PUBLIC        LockBit00
  C:007BH         PUBLIC        Pro00
  C:0115H         PUBLIC        RstPro00
  C:011BH         PUBLIC        Erase00
  C:0121H         PUBLIC        Read00
  C:011EH         PUBLIC        Write00
  C:0118H         PUBLIC        ReadSign00
  -------         PROC          RSTPRO00
  C:0115H         LINE#         9
  C:0115H         LINE#         10
  C:0115H         LINE#         11
  -------         ENDPROC       RSTPRO00
  -------         PROC          READSIGN00
  C:0118H         LINE#         16
  C:0118H         LINE#         17
  C:0118H         LINE#         18
  -------         ENDPROC       READSIGN00
  -------         PROC          ERASE00
  C:011BH         LINE#         21
  C:011BH         LINE#         22
  C:011BH         LINE#         23
  -------         ENDPROC       ERASE00
  -------         PROC          WRITE00
  C:011EH         LINE#         26
  C:011EH         LINE#         27
  C:011EH         LINE#         28
BL51 BANKED LINKER/LOCATER V5.03                                                      10/07/2003  00:07:48  PAGE 5


  -------         ENDPROC       WRITE00
  -------         PROC          READ00
  C:0121H         LINE#         31
  C:0121H         LINE#         32
  C:0121H         LINE#         33
  -------         ENDPROC       READ00
  -------         PROC          LOCKBIT00
  C:0124H         LINE#         36
  C:0124H         LINE#         37
  C:0124H         LINE#         38
  -------         ENDPROC       LOCKBIT00
  -------         PROC          PRO00
  C:007BH         LINE#         41
  C:007BH         LINE#         42
  C:007BH         LINE#         43
  C:0086H         LINE#         44
  C:009FH         LINE#         45
  C:009FH         LINE#         46
  C:009FH         LINE#         47
  C:00A2H         LINE#         48
  C:00A2H         LINE#         49
  C:00A2H         LINE#         50
  C:00A5H         LINE#         51
  C:00A5H         LINE#         52
  C:00A5H         LINE#         53
  C:00A8H         LINE#         54
  C:00A8H         LINE#         55
  C:00A8H         LINE#         56
  C:00ABH         LINE#         57
  C:00ABH         LINE#         58
  C:00ABH         LINE#         59
  C:00AEH         LINE#         60
  C:00AEH         LINE#         61
  C:00AEH         LINE#         62
  C:00B1H         LINE#         63
  C:00B1H         LINE#         64
  C:00B1H         LINE#         65
  C:00B1H         LINE#         66
  C:00B1H         LINE#         67
  -------         ENDPROC       PRO00
  -------         ENDMOD        AT89C51PRO

  -------         MODULE        ?C?ULCMP
  C:00F8H         PUBLIC        ?C?ULCMP
  -------         ENDMOD        ?C?ULCMP

Program Size: data=33.0 xdata=0 code=295
LINK/LOCATE RUN COMPLETE.  0 WARNING(S),  0 ERROR(S)
